:020000040800F2
:10000000500A0020D5000008E3000008E5000008C1
:1000100000000000000000000000000000000000E0
:10002000000000000000000000000000E7000008E1
:100030000000000000000000E9000008D90D0008E1
:10004000ED000008ED000008ED000008ED000008DC
:10005000ED000008ED000008ED0000080D040008A8
:10006000ED000008ED000008ED000008ED000008BC
:10007000ED000008ED000008ED000008ED000008AC
:10008000ED0000080000000000000000ED00000886
:1000900000000000ED000008ED000008ED00000881
:1000A00000000000ED000008ED000008ED00000871
:1000B000ED000008ED000008ED0000080000000061
:1000C0000348854600F054F800480047C512000870
:1000D000500A0020064880F30888064880470648F2
:1000E0000047FEE7FEE7FEE7FEE7FEE7FEE700006B
:1000F000500A0020DD0D0008C100000830B50B4695
:10010000014600202022012409E00D46D5409D42F1
:1001100005D31D469540491B254695404019154677
:10012000521E002DF1DC30BD03460B439B0703D06C
:1001300009E008C9121F08C0042AFAD203E00B78AC
:100140000370401C491C521EF9D27047D2B201E024
:100150000270401C491EFBD270470022F6E710B522
:1001600013460A4604461946FFF7F0FF204610BD25
:10017000064C0125064E05E0E36807CC2B430C3CFA
:1001800098471034B442F7D3FFF79EFF901400084D
:10019000B014000800F0BCF8FCE7000010B500F057
:1001A0007FF8012810D0094C207801280CD100F0EC
:1001B000F3FEA26861688918FF31F531884203D3E4
:1001C0000020207000F0C8F810BD0000D80000200A
:1001D00010B50D4C0120207000F0DEFEA06000F094
:1001E0005FF801280FD0207801280CD100F0D4FE50
:1001F000A26861688918FF31F531884203D3002075
:10020000207000F0A9F810BDD800002010B500F053
:1002100087F800F071F800F0CDFE00F0EFFC00F080
:1002200033F8FFF7D5FF10BD10B500F071F800F0FE
:10023000DDFE00F03FF8FFF7B1FF10BD7047000092
:1002400007480078002805D0012805D0022805D0ED
:10025000032803D0402070470820704700207047D3
:10026000E400002007480078002805D0012805D0C8
:10027000022805D0032803D040207047082070478B
:1002800000207047E400002010B500F0BDFE00F033
:10029000D9FC02490020087010BD0000E4000020D5
:1002A00010B5002400F0BEFE002800D00124204636
:1002B00010BD000008B56946064800F0F9FC0128A9
:1002C00007D105490020087068460178014800F010
:1002D000B1FE08BD78010020E400002010B5054AF9
:1002E0001278002A02D1C9B200F02AFD00F0D4FF32
:1002F00010BD0000E400002010B500F001F810BDB2
:1003000010B5024800F04AFC10BD0000B80B000018
:1003100010B500F001F810BD10B500F045FC10BD9F
:1003200010B500F001F810BD72B6704762B67047A4
:1003300070B50446501E0D4686B2002A0AD02878B1
:100340002070641C6D1CFFF7E3FF3046761EB6B2CA
:100350000028F4D170BD000070B500F053FC0028F7
:100360002FD000F031F800282BD0FFF767FF154899
:1003700081690122920391438161C169D200914355
:10038000C16100F02BFE0121084600F04FFC012561
:100390006D0700F02FFC0446BF2620782870641CEF
:1003A0006D1CFFF7B5FF3046761EB6B20028F4D1BB
:1003B000032000F03DF800F01DFC4468FFF7B6FF95
:1003C000A04770BD0010024010B509200121C006F1
:1003D00000F02AFB002801D0002010BD012010BD34
:1003E000094900230B61C00048618B610520086149
:1003F0000869C20701D0C003FAD508694008400067
:1004000008618B617047000000E000E010B5092032
:100410008021C00600F00FFB0120C00300F002F8AD
:1004200010BD000001494861704700000004014010
:1004300003490A689208920002430A60704700006C
:100440000000014000B507490A6902231A430A6106
:1004500048610869402210430861034800F066F8CB
:1004600000BD000000200240FF0F000002480169AB
:10047000802211430161704700200240F0B50B4E0D
:10048000044630690D4601273843306121800F2032
:1004900000F04CF8042807D13169280C3943316148
:1004A00060800F2000F042F8F0BD00000020024004
:1004B000F8B5064604460D46C00700D0FEE7012009
:1004C000C002FFF71BFE8646002900D0FEE7002190
:1004D000002818D908466843841901208446002260
:1004E000680810D06F085000205A094B984206D176
:1004F000521C92B29742F6D86046002803D1491C9C
:1005000089B28E45E6D88E4500D100242046F8BD3C
:10051000FFFF000003480249416003494160704702
:100520002301674500200240AB89EFCD10B4124B88
:100530000246D868C00701D001200AE0D868400709
:1005400001D5022005E0D868C00601D5032000E0EF
:100550000420FF21521E491EFDD1012801D1002A8D
:10056000E7D119697724A14319613421D960002AA0
:1005700000D1052010BC704700200240F8B50446A9
:10058000480A40021646009022681F460D46501C3D
:100590000BD100992046CB054DD1914205D00122C7
:1005A00001605202201DFFF7C3FE216800988142BE
:1005B00005D00146204600F01FF904003BD020681A
:1005C000281A051900982D1DFF30FF3002300090C9
:1005D000FFF79EFE281B01214902001F884222D3FB
:1005E0001648009D844201D1154C0AE01548854209
:1005F00002D1124C054604E0204600F071F90028B3
:1006000003D020462946EA0501D0002408E002680C
:100610008A4205D0012201605202201DFFF788FEA8
:10062000002C08D0251D307828706D1C761C7F1E8C
:10063000CED10120F8BD0020F8BD00000804002044
:10064000040200200018000810B50A480068401C89
:1006500004D0084800F044F9002809D00648006892
:10066000401C04D0044800F03BF9002800D00120D1
:1006700010BD00000804002004020020F8B5054663
:1006800043480C46411B601E814216D3284600F0A9
:1006900085F806462819401E00F080F8FF2E0CD081
:1006A000FF280AD004460125A64200D90025032EC2
:1006B00001D3102C03D9002567E00020F8BD002DE0
:1006C00063D037460026FFF723FE0C203146414316
:1006D00030480918097AB94204D10C214E43014629
:1006E0008E5905E0761CF6B20E2EECD30026F643AA
:1006F0000027FFF70DFE0C20394641432548091815
:100700000A7AA24204D10C214F430146CF5905E099
:100710007F1CFFB20E2FECD30027FF430094002470
:10072000FFF7F6FD0C201B4960434018017A009842
:10073000814205D10C20444316482018406804E04B
:10074000641CE4B20E2CEBD300203818401E801B32
:1007500080014030040CFFF7DDFE0027002C12D989
:10076000FFF7D6FD0C48864206D23046FFF76AFEF8
:10077000042801D0002506E0012080027F1C3618E5
:10078000BFB2A742ECD3FFF771FE2846F8BD0000C8
:10079000FFFF0008E813000800F0000870B50546E8
:1007A00000240C4EFFF7B4FD21460C204143705845
:1007B000A84209D8891949684018A84204D90C20D0
:1007C0004443A019007A70BD641CE4B20E2CE9D336
:1007D000FF2070BDE81300080048704700180008AB
:1007E00000200349C04308600249086070470000C8
:1007F000040200200804002070B5044610480D468D
:10080000844201D10F4C0AE00F48854202D10C4CC2
:10081000054604E0204600F063F8002804D0204696
:100820002946EA0501D0002070BD02688A4205D041
:10083000012201605202201DFFF77AFD204670BDA3
:100840000804002004020020001800080C480B4A8D
:1008500043680168591883685918C36859180369AF
:1008600059184369806959184018064909680818D9
:10087000106001D00020704701207047E800002080
:1008800000180008C018000870B5044610480D464E
:10089000011B681E1646814214D32046FFF77EFFD7
:1008A000FF280FD06019401EFFF778FFFF2809D0FE
:1008B000600A0849400288422B463246214603D14D
:1008C000054802E0002070BD0448FFF757FE70BDE8
:1008D000FFFF0008001800080804002004020020A0
:1008E000F8B50546012000902868FFF757FFFF285C
:1008F00010D0FFF70FFE00242868A1004618481901
:100900004768FFF705FD39463046FFF7B7FD042875
:1009100005D101E00020F8BD3068B84202D00020C7
:10092000009002E0641C802CE6D3FFF79FFD009846
:10093000F8BD000008B5002000900E480168491C71
:1009400015D0826841685118C2685118026951185F
:10095000426951188269C06951184018C043401C4F
:1009600000906A4604210448FFF78EFF08BD01206D
:1009700008BD000008040020C0180008F0B4CA78C0
:1009800013071B0FD20601D58A7813430022940661
:10099000240E0E88012595402E4207D005680F26AB
:1009A000A640B5431E46A64035430560521CD2B250
:1009B000082AECD30A88071D120A944600229406DE
:1009C000240E012595406646354207D03D680F2626
:1009D000A640B5431E46A64035433D60521CD2B2E8
:1009E000082AECD3CA78282A07D0482A03D10269FA
:1009F00009880A430261F0BC7047426909880A43CA
:100A00004261F0BC70474B0710B4DB0E082901D2DD
:100A1000203000E024300F249C4001689A40A1431C
:100A20001143016010BC70478068084000D001206D
:100A3000704741617047016170470021C9430180DF
:100A4000022181700421C170704710B500F020F8B8
:100A500000F032F800F058FC0921CC0601222046B3
:100A6000FFF7D1FF01220A212046FFF7CCFF606883
:100A7000F021884360606068902108436060606A8C
:100A8000102108436062606A09010843606210BD7A
:100A90000848416901225204114341610920C006FE
:100AA0000168090909010160016808221143016018
:100AB0007047000000100240F8B501214C042046A8
:100AC00000F0A8F801218D04284600F0A3F80121C8
:100AD000204600F09FF80121284600F09BF8684668
:100AE000FFF7ABFF082168460180012585701024BF
:100AF000294EC47069463046FFF740FF0821304652
:100B0000FFF799FF6846FFF798FFFF21023168461B
:100B100001808570C47069463046FFF72FFF96212B
:100B2000684601808570C4700924E4066946204641
:100B3000FFF724FF6846FFF780FFE903684601805E
:100B40004821C17069462046FFF718FF0221204660
:100B5000FFF76FFF04212046FFF76BFF6846FFF7A2
:100B60006CFF4021684601800421C170694630460F
:100B7000FFF704FF10212046FFF75BFF802120468E
:100B8000FFF757FF01213046FFF753FF2902304698
:100B9000FFF74FFFF8BD00000004004801494880FE
:100BA00070470000D000002010B500F0F5F9094CA6
:100BB000616888420DD300F0EFF9618840186060E9
:100BC0002078411C2170082803D908210248FFF72A
:100BD00030FF10BDD00000200004004810B5FFF722
:100BE000A9FE002801D0FFF72FFD10BD10B5FFF7BB
:100BF00045FD10BD10B5FFF7EFFD10BD10B5FFF7B7
:100C0000EFFD10BD10B5FFF721FE10BD10B5FFF7C9
:100C10003BFE10BD044A0029516901D0014300E0A8
:100C2000814351617047000000100240044A0029CE
:100C3000916901D0014300E0814391617047000058
:100C40000010024070B517488169012292031143D8
:100C50008161C1681143C160C1689143C160124C98
:100C6000A06940084000A061A06918210843A06164
:100C7000E06930210843E0610C48E1210068490344
:100C80000546FFF73BFA2062E12149022846FFF7BB
:100C900035FA0007000F6062A06901210843A061D6
:100CA00070BD00000010024000380140C800002064
:100CB000F3B5204C84466278002502201E4F1F4960
:100CC00081B0002A19D02378BE68CA18521CB60712
:100CD00025D57E68167078615B1CDAB222700878C0
:100CE000904223D16046491CFFF722FB65700298B1
:100CF00021780170012003B0F0BD104AB96889075E
:100D000014D57968C9B211707861491E3F290DD890
:100D100000F042F9606025700120607006E000F08C
:100D20003BF961686431884200D96570002003B0E6
:100D3000F0BD0000EC000020003801400C0600204F
:100D4000F3B581B00E46402903D9752119A0FFF7EC
:100D500021FA204F3E6000F01FF90446B8680A34BB
:100D6000C00708D1FFF7D4FA00F016F9A04202D864
:100D7000B868C007F6D00024002E18D9FFF7C8FACB
:100D80000198005D386000F007F90546B8680A353B
:100D9000C00708D1FFF7BCFA00F0FEF8A84202D85D
:100DA000B868C007F6D0641CA4B2B442E6D303B05E
:100DB000F0BD0000536F757263655C4F70656E42E5
:100DC0004C545C706C6174666F726D5C727332331C
:100DD000322E63000038014070470000F0B56349CF
:100DE00087B00A68012002430A604A68604B1A40D3
:100DF0004A600A685F4B1A400A600A6883049A4393
:100E00000A604A68C3231B049A434A600A685A4B23
:100E10001A400A609F2212048A600A6802430A602C
:100E200008688007FCD55648544D564A056010683E
:100E30001023184310601068C008C0001060022022
:100E40000090106802231843106048684E4A104012
:100E500048604868902210434860486848604348AA
:100E600041680215114341604848069002A8059068
:100E700003A8019000202E4607460490F8B20024F3
:100E800000900698611C4843791CFFF737F9A84287
:100E900001D9401B00E0281A864205D9064605986C
:100EA0000470019900980870002E08D0641C402C32
:100EB000E7D30498002802D17F1C042FDED33448E6
:100EC00001698908890001610169490849000161D6
:100ED0006946097B254C4907490F01916946097A02
:100EE0004906490E0091E16982051143E1610169FA
:100EF000284A114001610099019A09041202114324
:100F0000026911430161206801210906084320603C
:100F10002068800103D400BF20688001FBD5606891
:100F2000800880006060606802210843606060683B
:100F30000007800F022805D000BF60680007800FFF
:100F40000228F9D10120FFF74BFA61681020814394
:100F500061600120FFF744FA606880218843606087
:100F60000120FFF73DFA07B0F0BD0000001002407D
:100F70000CC0FFF8FFFFF6FEFFFF8F0000A24A043F
:100F8000C8000020002002400FC0FFFF00127A00BE
:100F900040100240FFF800FF04480069C103044804
:100FA00002D50168491C01600068704700E000E05C
:100FB000F400002006480021016141618161054A79
:100FC00042618161052202610348016070470000AF
:100FD00000E000E03F190100F40000200249002079
:100FE000086148618861704700E000E004480069DA
:100FF000C00303D503480168491C01607047000025
:1010000000E000E0F4000020044A002111700448D0
:101010009164C1708180917051707047B801002057
:10102000F801002002480078002800D00120704715
:10103000B8010020F8B505460078FF26924CFF283D
:1010400010D0924F397801297ED1F4284CD02CDC75
:10105000D0287AD020DCC92878D0CC2877D0CF28E7
:1010600076D1E9E0894D0020687001272F70EE707D
:10107000102129716871FFF7E3F8A871FFF7F2F802
:10108000E871FFF7EFF8000A28726F72AF7208205C
:10109000A080FFF7B3FDE2E07C49D1288A6C76D0CE
:1010A000D22875D0F32853D135E0F5380A284FD22D
:1010B00001007944097949188F44042ACBCBCB4EDF
:1010C000CB595F6BFFF7BCF86A78401E90427DDB1E
:1010D000381DB96CFFF72CF9FE706978B86C4018B0
:1010E000B8646878401CABE0FFF7AAF86978401E46
:1010F00088426BDB6968B9646A78381DFFF718F9B4
:10110000FE706978B86C4018B8646878401C97E045
:10111000FE70686851E05D48C6706F68C01D0025AC
:10112000164600907F1E07D33078761C4019C5B252
:10113000FFF7EEF87F1EF7D20098012105605348B3
:1011400001710021417104E09DE039E026E079E081
:101150007FE08171082073E0FE704D48B864002084
:1011600038717871B8714B4807214160F2E7FE2170
:101170000020F9703871022062E0FE7000203871A2
:1011800079787971B871F8713872062058E04AE0C0
:101190003DE0002038707870FE704BE0FFF750F8AB
:1011A000411E6A1CB86CFFF731FD002829D0FE7083
:1011B000FFF746F8B96C401E4018B8643AE005E005
:1011C000FFF73EF86978801E884205DAFE2122206A
:1011D000F9703871022033E0FE700120A080697838
:1011E00000290AD0AA1CB86CFFF710FD002808D00F
:1011F0006978B86C4018B86431E0FFF7EFFC00285C
:101200002DD1FE213120F9703871022018E0FE70D6
:1012100000253D717D71FFF713F8B871FD713D72C6
:101220007D7207200CE010466968FFF7DFFC00289C
:10123000E7D0FE70012003E0FFF78EF8FE7001207A
:10124000A0800CE0FE213120F97038710220A080CE
:1012500005E0FE212020F97038710220A080E0789E
:10126000012806D10949FE221020CA700871022007
:10127000A0800421615E002905DD0120E0700548A1
:1012800089B2FFF72BF8F8BDF8010020B801002063
:10129000E0130008BB01002001480021C170704725
:1012A000F801002002E008C8121F08C1002AFAD184
:1012B00070477047002001E001C1121F002AFBD1D6
:1012C00070470000FFF7C1FBFEF7A0FF00260C4CA3
:1012D0000C4D2670012701210920C903C006FFF724
:1012E000A3FB002803D02E70FEF79EFFF3E72878BB
:1012F0000028F9D12F702078401C2070F4E70000FE
:10130000C4000020CC00002070B540212F48FEF71B
:1013100024FF2F4E40242D4D21463046FFF7C8F8BC
:10132000002809D0B04201D12A4901E001464039E4
:1013300022462846FEF7F8FE2449002205200B88A5
:10134000891C9A180346401E92B280B2002BF6D137
:101350001E4881898A421ED101881F4A91421AD1B2
:101360004189002917D141880924E4061B4D002931
:1013700012D001291DD0022901D003290BD18021CF
:101380002046FFF758FB01212846FFF752FB1021AA
:101390002046FFF74EFB70BD80212046FFF74BFB38
:1013A00001212846FFF747FB10212046FFF743FBAA
:1013B00070BD01212846FFF73EFB80212046FFF744
:1013C00038FB10212046FFF734FB70BDF8000020E9
:1013D00000F80008C0FF0008FBAA00000004004855
:1013E0004F70656E424C5400001800080008000061
:1013F00003000000002000080008000004000000B6
:101400000028000800080000050000000030000867
:101410000008000006000000003800080008000076
:10142000070000000040000800080000080000005D
:1014300000480008000800000900000000500008F3
:10144000000800000A000000005800080008000022
:101450000B00000000600008000800000C00000005
:1014600000680008000800000D000000007000087F
:10147000000800000E0000000078000800080000CE
:101480000F00000000800008008000001000000035
:10149000B0140008C800002030000000A4120008AA
:1014A000E0140008F800002058090000B4120008F9
:1014B00000A24A040000000000000000000000003C
:1014C0000000000000000000000000000400000018
:1014D000000000000000000000000000000000000C
:04000005080000C12E
:00000001FF
